:100000000030660086000030650085009C200514E5
:1000100085150515412021308F003C20C5308F000B
:100020003C2013308F003C2020308F003C200930D2
:100030008F0087203C209C209C209C209C20083006
:100040008F003C209C209C200C308F003C204030B6
:100050008F003C2080308F003C201F308F003720E5
:1000600005308F00372007308F0037202D280514EA
:10007000851145208515003405108511452085150D
:10008000003485109C208514003406138F1B8617BE
:100090008F1F8613A9200617A92006130F1B86178A
:1000A0000F1F8613A9200617A92006138F1A86177B
:1000B0008F1E8613A9200617A92006130F1A86176C
:1000C0000F1E8613A9200617A92006138F1986175D
:1000D0008F1D8613A9200617A92006130F1986174E
:1000E0000F1D8613A9200617A92006138F1886173F
:1000F0008F1C8613A9200617A92006130F18861730
:100100000F1C8613A9200617A92006130034861396
:1001100006308E0054308C0008308D000514851197
:1001200006130000000006178D0B902885158C0B18
:100130008C288E0B8A28003407308E0032308C00D9
:10014000FA308D008D0BA2288C0BA0288E0B9E28D8
:10015000003420308C0040308D008D0BAD288C0B8E
:04016000AB28003494
:02400E00F93F78
:00000001FF
